:020000020000FC
:100000009EC118951895EDC718951895EFC71895C6
:100010001895DAC718951895189518951895189584
:100020001895189518955F9BFECF4CB108954DE03B
:100030005D9BFECF4CB90895332770FD05C03FB9D5
:10004000779BFECF3FB108950F931F932F9309E045
:100050000EBD2227726071FDFECF2F911F910F916F
:1000600008953B2DEADF3A2DE8DF08953991E5DF69
:10007000019780309807D1F708953091BB02DDDFFA
:100080003091BC02DADF3091BD02D7DF3091BE0281
:10009000D4DF089500270DB9BB98C59864FD02C050
:1000A000C29801C0C29AC198B998BD98BA980895EB
:1000B000BA9A64FD02C0C29A01C0C29802E095D00B
:1000C000C398C598C198BB9ABD9AB99ABC9800E5E7
:1000D0000DB964FD02C0C29801C0C29A02E085D089
:1000E000C19A64FD02C0C29A01C0C29802E07DD0EC
:1000F0008BE09927B3D0EAE4F1E00591073220F4D0
:10010000011711F03396F9CF05910023B9F4059149
:100110001EB11E7F102B1EB90CEF1DB110230591CF
:10012000102B1DB963FF07C075FF05C057FD03C045
:1001300051FD01C06A9A6E9A7E7F089505911591CE
:100140001BBD0ABD6E987160089500000101010099
:100150000102020000030301800026019903FF0150
:10016000001830EF6ADF68DF67DF66DF30FDF9CF48
:100170000895C1983AEA61DF30E65FDF5DDF5CDF5A
:100180005BDFC19A30FFF5CF0895C895002021F0BC
:10019000402D4EDF3196F9CF0895C895002021F00B
:1001A000402D46DF3296F9CF0895C895002021F002
:1001B000501519F03296F9CF08940895C89500208B
:1001C00041F0501511F03296F9CF3196C895502C68
:1001D000D52C0895C895002039F0501511F03296AD
:1001E000F9CF3196C895402C089503950A9509F4E6
:1001F00008950F930CE005BD05B502FDFDCF0F91ED
:10020000F5CF1BDF3D2F19DF3C2F17DF0895C59A6F
:1002100070FF6E9802E0E9DFC59870FF6E9A02E009
:10022000E4DF08955523B2F030E207DF3D2F05DF0C
:100230003C2F03DF01DF432FFBDE55234AF038E27A
:10024000FCDE3D2FFADE3C2FF8DEF6DE432FF0DE3B
:10025000219608953D2F3ED03160E9CFE199FECF40
:100260008EBB9FBBE09A1DB30895E199FECF8EBB74
:100270009FBB1DBBE29AE19A0895552322F030EA14
:10028000DCDE3D2F05C0573859F03D2F23D03560B7
:10029000D4DE3C2FD2DED0DE432FCADE2196089575
:1002A0000F910F9149C3552322F030ECC6DE3D2F4C
:1002B00005C0573861F03D2F0DD03660BEDE3C2FB3
:1002C000BCDE342FBADE0AE090DF219608950F914C
:1002D0000F9132C3330F330F330F18F4573809F42B
:1002E000346008953DE4A9DEA7DE342DA6DEA4DE49
:1002F000089514E0AD98AC98AB9AAA98A99A0AEF21
:1003000074DFAD9AAC9AAB98AA9AA9980AEF6DDF00
:100310001A9581F708956061AC9A10FD08956F7E7B
:10032000AC98089500EF702E01E0602E746004E038
:1003300003BF0895002703BF7B7FAB9A08950FE5A5
:1003400014E00DBF1EBF00E1502ED52C1FEF12BBD5
:100350001FEF18BB1FEF15BB1EE314BB12E011BB50
:10036000772766276FBD6093B802599803E009B9F3
:1003700008E10AB901E909BF03E703BD08E00EBDC2
:1003800008E005BD002703BF0DBD0CBD7894B1DFAB
:1003900099278DE063DFBFDF5F9903C072FFC2DF83
:1003A000FBCFC8DF40DE4B3119F04335A9F766C0FB
:1003B000ECE8F1E00BE1F02E019335DE4B3121F456
:1003C000E3944E1539F04DC0433521F4E3944E15B6
:1003D00009F054C06860E42E4193F42624DEB42F63
:1003E000F426002701931FDEA42FF42601931BDEC1
:1003F0004E3091F6F4264193C0E6D0E014DE4993E6
:10040000F4260E91A030D1F7B030C1F70CDEF4160F
:1004100009F0C2CFA0E6BB270C91019300E0008356
:10042000E6E2F1E10591002309F4B6CF1C91101723
:1004300011F03396F7CF259105911591F8010995A3
:10044000ECE8F1E0FF244191F426F2DDEA17FB0726
:10045000D1F74F2DEDDD00919101073009F09CCFD0
:10046000D2CB677FE0DD4B31E1F308C065D25F9905
:1004700003C072FF57DFFBCF5DDFD5DDECEAF0E1B3
:100480000591002399F3401711F03396F9CF259188
:1004900005911591F801222331F0ABEBB2E0C3DDF9
:1004A0004D932A95E1F76E7F099560FD81CFDFCFEF
:1004B000ABEBB2E04C91542F152F80E19927D5DE9C
:1004C000AC986F7E552312F06061AC9AE2E6F0E1E1
:1004D00075DE0FEF402EE2E4F0E17CDE6260E2E4E4
:1004E000F0E163DE28F0E2E6F0E15FDE08F06D7F28
:1004F0009ECD61600895E4EAF0E147DE0895ECE9FD
:10050000F0E143DE0895E0EAF0E13FDE0895E2E441
:10051000F0E143DEE2E6F0E140DE40E089DD08950F
:1005200043E586DD089549E583DD0895EAE7F1E1D5
:100530002CDE4AE07DDD7BCD49E57ADD40E078DDEB
:1005400040E876DD0895AD9A72CDAD9870CD61FF2B
:10055000F3C1AEDDAD9802E348DE3CEA6EDD33E583
:100560006CDD503280F0552372F020E265DD3335CA
:1005700061F030E062DD4BDE3CEA5FDD33E55DDDFE
:100580002A95A1F702C030E058DD552312F030E083
:1005900054DD04E02ADE4BCD61FFCEC130E4132EE2
:1005A00055231AF04ADD3D2F03C03D2F93DE326004
:1005B00044DD3C2F42DDABEBB2E03C91C32E3DDD90
:1005C0008C2E9D2E55230AF421966BC161FFB4C178
:1005D000552382F038E4132E30DD3D2F2EDD3C2FE5
:1005E0002CDDABEBB2E03C91C32E27DD8C2E9D2E93
:1005F000219657C1A1C161FF9FC16F7DABEBB2E0F6
:100600000D91002309F098C10D91013808F094C1B3
:10061000802F902F0C910093B902BB27A0E603DD39
:100620004D938A95E1F7A0E64091B902463441F036
:10063000453409F081C14D9136DE9A95E1F7F7CC4A
:100640001E01D52CE2E6F0E1B0DD08F42EC030E466
:10065000032FD7DD3D9165FD07C0341529F0606299
:10066000102EC32E8C2E9D2EE8DC38E4032FC9DD1E
:100670003D9165FD07C0341529F06062102EC32E30
:100680008C2E9D2EDADC21969A959A95DA9411F0AB
:100690009923E9F63CE4D1DC332DCFDC322DCDDCDF
:1006A00030E0CBDCD52C6F7D27C15523EAF0CD900F
:1006B000C39449F0CA9430E4132EA3DD3C2DBDDC75
:1006C0008C2E9D2EF3D09A95CD90C39449F0CA9468
:1006D00038E4132E96DD3C2DB0DC8C2E9D2EE6D01A
:1006E00021969A9511F7A3CC3D2FF4DD3260A5DC5D
:1006F0003C2FA3DC3D91C32EA0DCEFCF61FF1CC1DA
:100700005523B2F038E299DC3D2F97DC3C2F95DC85
:1007100093DC432F8DDC55234AF030E28EDC3D2FF5
:100720008CDC3C2F8ADC88DC432F82DC2196089508
:100730003D2FD0DD3160E9CF61FFFEC0ABEBB2E011
:100740009D918D912C91263439F0253409F0F4C017
:1007500094DD0197E9F70895552322F063DD0297B0
:10076000E9F708955FDD0197E9F7089561FFE4C0B7
:10077000ABEBB2E0DD91CC915ACC61FFDDC0ABEBCD
:10078000B2E04C9190DD53CC61FFD6C076DD089588
:1007900061FFD2C064FD02C0C29801C0C29A12E0DB
:1007A00011BBAD9A44CC61FFC7C03CEA46DC55237F
:1007B00012F030E842DC34E040DC30E03EDC08E2BD
:1007C00014DD35CC61FFB8C0ABEBB2E03CEA35DC00
:1007D00055238AF05E3539F03C913670306E2DDC51
:1007E00030E02BDC0CC030EE28DC30E026DC3C9125
:1007F0003C6F23DC06C03C91307E37601EDC30E06D
:100800001CDC0AE0F2DC13CC61FF96C055233AF001
:1008100012E006D011E004D010E002D008958CC0A0
:1008200030E30BDC30E009DC312F07DC05DC432F43
:10083000FFDB089561FF80C03CE4FFDB392DFDDB69
:10084000382DFBDB30E0F9DB57C061FF75C0ABEB47
:10085000B2E03D91F2DB3D91F0DB3C91EEDBECDB75
:10086000432FE6DB02E3C1DCE2CB61FF65C0ABEB0B
:10087000B2E03D91E2DB3D91E0DB3D91DEDB3D917D
:10088000DCDB432FD5DB02E3B0DCD1CB61FF54C00E
:1008900038E5D3DB3327D1DBD0DBCEDB432FC8DB1E
:1008A000C6CBE2E6F0E181DC10F0C1CB646044200D
:1008B000E9F0C414D9F0212D2F702062122E2227C6
:1008C000552322F0312DB9DB392D03C0392D02DD3E
:1008D0003160B3DB382DB1DBAFDB0C2D552312F4C7
:1008E00030780078301721F02A9551F70AE07DDC46
:1008F00062FF9DCB6B7F08955134A9F05332D1F044
:1009000065FF11C0212D2F702062122E2227312D5C
:1009100094DB392D92DB382D90DB8EDB3C1529F0F2
:100920002A9509F0F4CF02E360DC1E01992309F057
:100930008ECE7DCB16DCF9CF4FE37ADB08950590A0
:100940000D920A95E1F7089501900D920A95E1F74D
:1009500008950BE000938F01A3E9B1E0E4E6F9E02C
:1009600009E0EDCF084156524953505F320002E092
:1009700000938F01A3E9B1E0209161001091620022
:100980002F3931F0283919F48BE099276EDC08955E
:100990001093B802089503E000938F01A4E9B1E039
:1009A000209161001091B8022F3951F099278FEFF3
:1009B000839554DC112321F083952117C9F74EDC70
:1009C000109393010895A1E6B0E00D916D7F6B7FC8
:1009D00007FF02C0626086DC4D903D902C907064F1
:1009E00002E000938F01A3E9B1E00895F9CFAD983B
:1009F0006A987F7D8DE0992731DC212F11270091A6
:100A0000660004FD1160211330DC85DC552706FDEE
:100A10000EC07062502F51FF0AC04ADBC1983AEAFB
:100A20000CDB3CEA0ADB33E508DBC19AD9CF40DBBB
:100A300000916100DADB2091640030916800FDDAFA
:100A400000916500D2DB30916900F7DA0091650012
:100A5000CCDB30916A00F1DA75FF02C057FD24C08B
:100A6000132F00916500C1DB30916B00E6DA009135
:100A70006500BBDB00916700033061F0043079F062
:100A8000002389F0C4DB2A95C1F600EC00939201A3
:100A9000AD9AA6CF009166000113F4CF04C0009177
:100AA00066000313EFCF9CCF05E09FDB99CFF2DA0E
:100AB000AD9A96CF75FF04C051FD20C057FD0FC001
:100AC000C3E6D0E084E09927D1DA009162000023E8
:100AD00021F40091610089DB83CF43DB81CF3CEAC5
:100AE000ACDA34E0AADAA8DA0FEF0093BA0231E008
:100AF000A4DAA2DAA1DA3323B9F372CFC1983AEAC1
:100B00009CDA3AE89ADAC19A34DB6ACF7F770FE051
:100B1000D02E75FF05C076FF03C07F7B220C331CEF
:100B2000F1018091620090916100AAE6B0E075FF4A
:100B30002BC057FDC8C05530D9F051FD0BC000E5A2
:100B400077FD02E50093650000E277FD02E2009385
:100B5000670018C0C1983AEA70DA00E577FD02E54F
:100B60000093650000E377FD08E3009367000AC087
:100B700000E577FD00ED0093650000E277FD00EBF6
:100B8000009367000AEAD02E2091630020FD3AC04E
:100B9000D29430916500D0FC38604FDA5F0161DAA1
:100BA0003D91032E4ADA22FD0AC023FF27C0D9DA7D
:100BB000D1FC319601978030980751F782C000919F
:100BC00068000015D9F00AEA0D1521F400916900BA
:100BD0000015A1F030916700D0FC38602EDA5F017B
:100BE00040DA2ADA00916800301749F30AEA0D1555
:100BF000F9F600916900301711F3DACF0091640023
:100C0000F4DAD6CF6F7D6F7BD29430916500D0FC43
:100C1000386013DA5F0125DA3D91032E0EDA25FFE5
:100C200012C065FD10C000916800001561F00AEA6D
:100C30000D1521F400916900001529F060624F0143
:100C4000D0FC01C06064D1FE04C0319611F461FD96
:100C5000646001978030980719F075FFD5CFDCCF1D
:100C600075FF03C051FD4FC008C027FF2AC0309157
:100C70006600E3D95101F5D9DFD925FF16C065FF1C
:100C800018C03091670066FF3860D7D95401E9D9A0
:100C9000D3D9009168003017A1F30AEA0D1521F4A9
:100CA00000916900301769F307C026FF02C059DAC6
:100CB00003C00091640099DA62FF03C0439412DB21
:100CC0006B7F1F018DCE3F2F05DB3260D0FE34607D
:100CD000B4D93E2FB2D93D91032FAFD93F2FFADAC5
:100CE0003160D0FE3460A9D93E2FA7D9A5D93027CD
:100CF00037FDF4CF319601978030980721F7E1CF87
:100D00000AE073DAF7CFC19A34DADBCF7F770FE0EE
:100D1000D02E75FF05C076FF03C07F7B220C331CED
:100D2000F101A3E9B1E08091620090916100039626
:100D300090938E0180938F01809162009091610069
:100D400075FF17C057FD34C051FD09C0553009F07B
:100D500009C000E377FD00EB0093630008C0C19871
:100D60003AEA6BD900E377FD02E3009363000AEAF5
:100D7000D02E20916300D294322FD0FC38605DD900
:100D80005F016FD959D93D93D1FE06C0319621F448
:100D900061FF02C04394A6DA01978030980719F0EA
:100DA00075FFE9CFEFCFC19A00E00D931F010895C1
:100DB0003F2F90DA3160D0FE34603FD93E2F3DD9CD
:100DC0003BD93D93319601978030980789F7EBCF57
:100DD00070680AEAD02EA4CE70680AEAD02EA0CF9E
:100DE00075FF40C051FD16C057FD09C03CEA25D92A
:100DF00030916400377E21D91FD91ED938C03CEA12
:100E00001CD9309164003093BA0264DA376015D986
:100E100013D92DC0C1983AEA10D934EE1BC075FF22
:100E200021C051FD0EC0009164000E7F009364004C
:100E30003CEA03D9309164003F71FFD8FDD8FCD85B
:100E400016C0009164000E7F00936400C1983AEAD6
:100E5000F4D831EEF2D8F0D8EFD830916400EDD864
:100E6000C19A05C0C1E6D0E084E09927FFD803E02D
:100E700000938F01A3E9B1E000E00D93089575FFA1
:100E800041C051FD06C031E2D8D8D6D8D5D8D4D883
:100E900008C0C1983AEAD1D831E6CFD8CDD8CCD85D
:100EA000CBD8C19A04E000938F01A3E9B1E03D9350
:100EB0003EC075FF27C051FD06C034E2BED8BCD885
:100EC000BBD8BAD8EECFC1983AEAB7D834E613E027
:100ED000E4CF75FF17C051FD0AC038E2AED8ACD8D8
:100EE0003091640052FD3063A8D8A6D8DACFC198FB
:100EF0003AEAA3D838E3A1D89FD8309164009DD8AE
:100F00009BD8CFCF04E000938F01A3E9B1E0C1E605
:100F1000D0E02991002775FF02C057FD0BC0399121
:100F20008CD80395021709F43D930430C1F700E013
:100F30000D930895109160001A3151F000916400F2
:100F40002227E8E5FFE0E00FF21F14911D93EFCF99
:100F50003091BA023D93EBCF1E720000A3E9B1E0DD
:100F600010916200C4E6D0E00091610080916300BE
:100F7000E8941123C1F0882359F0002309F4689400
:100F800033270EF0399159D80EF00A958A95A9F7B2
:100F9000002309F46894332716F039910A954DD847
:100FA0003D931A95A9F7002321F0399146D80A9567
:100FB000E1F700E00D9380916200992703969093EA
:100FC0008E0180938F0108950F9300E702BF6A940A
:100FD00031F47294AB9A70FCAB9804E6602E0F91DA
:100FE00018950F9308E005BD0F9118952223B9F0CD
:100FF000229520FD0DC0C59863FF189575FF1895C3
:1010000057FD189551FD1895110FB4991160189559
:101010000A9541F4312F7D7F08E00EBD189508E058
:1010200011272FE0331F10F4C39A01C0C398C59A4B
:1010300063FFEACF75FFE8CF57FDE6CF51FDE4CF60
:1010400018951300207F287F30FF34FF387F48FF3A
:101050004CFF51FF55FF56FF68FF6CFF86FF87FF6F
:10106000000023103A203B2041404340444045408B
:1010700046405E10604061406240634064406640AC
:1010800069206A2072407340744075407620772052
:1010900078407940652067204240000033370000E7
:1010A000313200004156522039313000540158028B
:1010B00053007B0256007F02760083027400870291
:1010C000700090027801A3027901A5025000A702E6
:1010D0004301E6026301CC0262009C024203FB0270
:1010E00052007E034102B6034401BD036400C40301
:1010F0004C00C8036500D3036C01E2037200460490
:10110000730004046D001A043A0325042E04350408
:10111000610093026900960267039C034500C803BF
:101120001B00790200000100A9040200B7040300BB
:10113000CB040400E3040500E3040600E304070015
:10114000F6041000F7041100570512005A051300A9
:101150008605140086061500E8061600EC06170042
:101160000F0718003F071900F0061A0059071B0067
:1011700069071C0082071D00AE07626970726F6705
:10118000202D204156522070726F6772616D6D651F
:101190007220696E2061677265656D656E74207777
:1011A000697468206E6F746573204156523931300E
:1011B00020616E6420415652303638200D0A566543
:1011C0007273696F6E20312E35202D20392E303507
:1011D0002E32303038200D0A687474703A2F2F7711
:1011E00065622E717569636B2E637A2F7275636BFE
:1011F0006C2F626970726F672F626970726F672EF1
:0612000068746D6C200013
:00000001FF
